:100000000C9435010C9458010C9458010C9458012F
:100010000C9458010C9458010C9458010C945801FC
:100020000C9458010C9465010C9458010C946105D2
:100030000C9458010C9458010C9458010C945801DC
:100040000C9406080C9458010C94C6050C945801A5
:100050000C9458010C9458010C9458010C945801BC
:100060000C9458010C94580100000000000000009E
:100070000000160455000103FF0300000300060002
:1000800000050006000700080009000A090109022E
:1000900001020103003000000000213D0200033D89
:1000A0000200213D0200213D0200213D0200213DD0
:1000B000020000000000000000000000000000003E
:1000C0000000000000000000000000000444FFFFEA
:1000D000FFFFFFFF0000FFFFFFFFFFFFFFFF00002C
:1000E0000004000001000000000000020000000009
:1000F0000000000000000000000000000000000000
:100100000000000A0A0A0A0B0A0A0A0A0A0A0D0C67
:100110000A0A0A0A0A0A0A0A0E0A0A0A0A0A0A0A3B
:100120000A0A0A0A0A0A0000000000000000000093
:1001300000000000000000000000000000000000BF
:1001400000000000000000000000000000000000AF
:10015000000000000000000000000000000000009F
:10016000000000000000000000000000000000008F
:10017000000000000000000000000000000000007F
:10018000000000000000000000000000000000006F
:10019000000000000000000000000000000000005F
:1001A000000000000000000000000000000000004F
:1001B000000000000000000000000000000000003F
:1001C000000000000000000000000000000000002F
:1001D000000000000000000000000000000000001F
:1001E000000000000000000000000000000000000F
:1001F00000000000000000000102060A09000000E3
:100200000000030C0D0700000000000000000000CB
:1002100000000000000000000000000000000000DE
:1002200000000000000000000000000000000800C6
:1002300000000000000000000000000000000000BE
:1002400000000000000000000000000000000000AE
:100250000000000000000000000000002313221234
:100260002111203633322524350011241FBECFEF53
:10027000D4E0DEBFCDBF11E0A0E0B1E0EEE0FBE2F4
:1002800002C005900D92A830B107D9F712E0A8E09E
:10029000B1E001C01D92A836B107E1F7E8E6F2E04F
:1002A0008AEA95E08193E030F907E0F30C94530279
:1002B0000C940000E091C201F091C301309719F055
:1002C0000995E82FFF27CF0108951F920F920FB6CF
:1002D0000F9211242F933F934F935F936F937F93CC
:1002E0008F939F93AF93BF93EF93FF9382E00E940E
:1002F0005A01FF91EF91BF91AF919F918F917F91A3
:100300006F915F914F913F912F910F900FBE0F9082
:100310001F9018958091B6019091B7010196909326
:10032000B7018093B60190E08091BB01882309F466
:1003300091E09093BB0183E00E945A0180910B01F0
:100340008823B1F4809167018F7780935D022091BB
:10035000670130916801220F232F221F330B922F48
:100360009F7090936502492F682F82EB0E94F604DC
:100370008AE090E008958091BE01882351F0809139
:10038000C00180958093C0018091C10180958093C8
:10039000C1018091C00180FF02C0439A01C043980F
:1003A00081FF02C0429A01C0429882FF02C0419A76
:1003B00001C0419883FF02C0409A01C0409884FF69
:1003C00002C02D9A01C02D9885FF02C02C9A01C051
:1003D0002C9886FF02C05F9A01C05F9887FF02C019
:1003E0005C9A01C05C988091C10180FF02C02B9A89
:1003F00001C02B9881FF02C02A9A01C02A9882FF6F
:1004000002C0299A01C0299883FF02C05E9A01C0E8
:100410005E9884FF02C05D9A01C05D9885FF02C0AE
:100420005B9A08955B98089530E08091BF0188231E
:10043000C9F021E0E7E6F1E0868197810196978394
:1004400086834F9724F0178216822087322F3996A1
:1004500081E0E63AF80781F37CF3332319F085E075
:100460000E945A018AE090E008950E943E0A84E1C9
:1004700090E008953B9A3A9A399A389A259A249AA4
:10048000579A549A239A229A219A569A559A539A8D
:10049000539852983D983C981092C0011092C10117
:1004A0000E94BB010895CFEFD4E0DEBFCDBFFF2493
:1004B000F894A89584B7877F84BF80916000886195
:1004C0008093600010926000789486EC91E00E9426
:1004D000B504519A0E9438080E94480C0E94420AB2
:1004E0001092B7011092B6011092B9011092B801A2
:1004F00081E08093BA011092BB018093BC0185E03A
:100500008093BD011092BE018CE090E00E94360FF6
:1005100080930001853511F00E94EB0F8BE090E095
:100520000E94360F80935C02833029F063E08BE0F9
:1005300090E00E94770F8DE090E00E94360F80934C
:100540000B018EE090E00E94360F8093BC018FE09B
:1005500090E00E94360F8093BD0181E190E00E94FF
:10056000360F982F91709093BE0182708093BF01D7
:1005700080E190E00E94360F80930A0199278F71E5
:100580009070809714F010920A0180910A01E7E6BA
:10059000F1E08283108617821682399691E0E63A5E
:1005A000F907B9F3B4F33B983A98399838982598F5
:1005B000249857985498239822982198569855989B
:1005C0005398539852983D983C9880910B019927E5
:1005D00089309105A9F08A30910524F4019702979A
:1005E000B0F405C0449799F489EF92E102C088E223
:1005F00091E19093C3018093C2010E943A020BC023
:100600008FE291E19093C3018093C20104C01092E4
:10061000C3011092C20180E00E945A0100E02BE564
:1006200032E04AE851E061E08FEA91E00E9445083B
:100630002BE532E044E152E06AE08EE592E00E9470
:10064000450801E02BE532E045E352E0602F84E508
:1006500092E00E94450864E170E085E190E00E942C
:10066000B913909368018093670166E170E087E1B8
:1006700090E00E94B913909371018093700168E13A
:1006800070E089E190E00E94B91390937A01809321
:1006900079016AE170E08BE190E00E94B9139093D8
:1006A0008301809382016CE170E08DE190E00E9413
:1006B000B91390938C0180938B016EE170E08FE110
:1006C00090E00E94B913909395018093940160E2A9
:1006D00070E081E290E00E94B91390939E018093B4
:1006E0009D0162E270E083E290E00E94B913909372
:1006F000A7018093A6010E94570D0E94760881E011
:100700000E945A010E945A130E94BC049093C50192
:100710008093C401009779F30E94CB0B813021F4C0
:1007200014BEE0E0FFE10994E091C401F091C5013D
:100730008081843E09F059C08181893009F055C01B
:10074000828199278F7790709695982F8827979513
:1007500087959093B9018093B801238133272F7730
:100760003070282B392B3093B9012093B801809138
:100770000B01882391F49091B8019F7790935D02CB
:10078000220F232F221F330B822F8F70809365023D
:10079000482F692F82EB0E94F6046091B801709196
:1007A000B901A091C401B091C501E7E6F1E08081F3
:1007B00091816817790799F4ED015C81513079F4E2
:1007C0008281282F332727FD30954E81842F99274A
:1007D0002817390709F0F52E4283178216823996B9
:1007E00081E0E63AF80719F314F3E091C401F091BF
:1007F000C5018081803B09F05EC0828199278F709E
:1008000090709695982F8827979587959093B90122
:100810008093B801218133272F773070282B392B13
:100820003093B9012093B80180910B01882391F492
:100830009091B8019F7790935D02220F232F221F82
:10084000330B822F8F7080936502482F692F82EBC4
:100850000E94F604C0E0D0E007E611E02091B80164
:100860003091B901F80180819181075F1F4F2817EE
:100870003907E9F4E091C401F091C501828185FF57
:100880000AC061E08C2F0E944A14882311F0E1E035
:10089000FE2E61E009C060E08C2F0E944A1488237C
:1008A00011F071E0F72E60E08C2F0E942414219645
:1008B000C830D1059CF2E091C401F091C50150818E
:1008C000523BC9F58281282F33272F70307036951F
:1008D000322F2227379527953093B9012093B801FD
:1008E000818199278F779070822B932B9093B901F8
:1008F0008093B801209167013091680182179307B6
:10090000D1F480910B018823B1F4809170018F772D
:1009100080935D022091700130917101220F232F8D
:10092000221F330B922F9F7090936502492F682FDF
:10093000852F0E94F604E091C401F091C5018081E9
:10094000853E19F4CF010E941E13FF2019F084E0A8
:100950000E945A011092B9011092B8018091C4010D
:100960009091C5010E94D10DC6CE90930D01809348
:100970000C010E942D05089580910C0190910D01AC
:100980000E940C070895EF92FF920F931F93CF934D
:100990007C01CEE210E001E06C2FC7010E942D0621
:1009A000833019F483E090E01BC0813011F400E043
:1009B000F3CF823088F3823011F4002369F7CB3112
:1009C00008F0C1501F5F193130F3E0910C01F09134
:1009D0000D01E657FF4F80818F5F808386E090E0B6
:1009E000CF911F910F91FF90EF900895CF93DF93D8
:1009F000CDB7DEB760970FB6F894DEBF0FBECDBFA0
:100A000089836A834B83CE0101960E94C304992790
:100A100060960FB6F894DEBF0FBECDBFDF91CF91C9
:100A20000895CF93DF93CDB7DEB760970FB6F894F4
:100A3000DEBF0FBECDBF89836A834B83622FCE0199
:100A400001960E942D06992760960FB6F894DEBF96
:100A50000FBECDBFDF91CF910895599A90930F01AA
:100A600080930E0180E98093C1008DE18093C400E2
:100A700080918100887F81608093810080E880BFC1
:100A80000895809184009091850090931201809345
:100A900011010197909389008093880081E08093F1
:100AA0001001B19A80916F00826080936F008091F5
:100AB00068008B7F80936800DA9A82E080936D00F3
:100AC00008951F920F920FB60F9211248F93809169
:100AD0006F008D7F80936F00109210018F910F90A7
:100AE0000FBE0F901F9018950F931F93CF93DF9316
:100AF000282F80911001882319F481E090E020C014
:100B00000091840010918500809111019091120153
:100B1000081B190BC0E0D0E0822F9927AA27BB271A
:100B2000BC01CD0120EE31E040E050E00E941C15F8
:100B3000DC01CB010817190710F0C1E0D0E0CE01AD
:100B4000DF91CF911F910F910895B19A90916F000D
:100B50009D7F90936F009927AA27BB27BC01CD01E9
:100B600020EE31E040E050E00E941C15DC01CB019A
:100B70009C018091110190911201820F931F90931B
:100B8000890080938800B19BFECF08951F920F9239
:100B90000FB60F9211242F933F934F935F936F9350
:100BA0007F938F939F93AF93BF93CF93EF93FF93D5
:100BB0008091C00084FF09C0E0910E01F0910F0107
:100BC000E957FF4F80818F5F80838091C00083FF52
:100BD00005C0809114018F5F80931401C091C600FD
:100BE00080911301882311F40E944105E0910E01C8
:100BF000F0910F01DF01A058BF4F8C91E80FF11D5C
:100C0000C0838F5F8C9387FD1C92FF91EF91CF91F2
:100C1000BF91AF919F918F917F916F915F914F9114
:100C20003F912F910F900FBE0F901F9018950E942B
:100C30004105599878948FE00E94A505599A0E9421
:100C4000410510921301E0910E01F0910F01E5575B
:100C5000FF4F80818F5F80830895CF92DF92EF9264
:100C6000FF920F931F93CF93DF93CDB7DEB72497F7
:100C70000FB6F894DEBF0FBECDBF6C01F62E0E94FA
:100C8000F006E82E4FEF00E0A82FBB279D01215072
:100C90003040121613065CF4F601E00FF11D80815E
:100CA00048270F5F802F992782179307ACF3AC0D6D
:100CB000BD1D11974C9388E38F1508F4F82E8BB364
:100CC00099279C012470307082FF03C00E94410567
:100CD00010C0890184E10E947405882311F4C801C1
:100CE00070C08F2D0E947405882331F481E090E05C
:100CF00068C082E090E065C00E9441050E1508F0D2
:100D00004FC081E08983F601E00FF11D80818A8365
:100D10001C82F89480918400909185009093120138
:100D200080931101489908C07894002311F30E9420
:100D3000170684E090E045C0599881E08093130144
:100D40001B828B818830D8F41A818981182309F09D
:100D500011E08B818F5F0E94A5058C81882311F0A3
:100D6000489BE5CF112311F0599A01C059981C8373
:100D70008981880F89838B818F5F8B83E2CF89E0A4
:100D80000E94A5058C81882311F0489BD0CF599AE9
:100D900078948AE00E94A505489BC9CF0F5FAECF2B
:100DA0000E94410510921301E0910E01F0910F0194
:100DB000E857FF4F8081918101969183808383E082
:100DC00090E024960FB6F894DEBF0FBECDBFDF9142
:100DD000CF911F910F91FF90EF90DF90CF900895EA
:100DE000FC0180819927807690708036910511F4FE
:100DF00081810AC0808199278076907024E0959542
:100E000087952A95E1F78E5F992708952CE8FC01D4
:100E100011922A95E9F70895BF92CF92DF92EF924F
:100E2000FF920F931F93CF93DF93EC01FE01EF57D7
:100E3000FF4FC058DF4F90818881C058D04098172D
:100E400009F4D5C09081FE01E90FF11DB080B7FE15
:100E50002AC0DE01AE57BF4F8C91891731F0FE01D9
:100E6000E957FF4F80818F5F80839C93CD57DF4F81
:100E70008FEF8883C358D040FE01EC57FF4F8B2D76
:100E80009927807690708036910539F074E09595B9
:100E900087957A95E1F78E5F01C080E08083882393
:100EA00009F465C008C0FE01EC57FF4F808188231C
:100EB00009F05DC0B082AE014E575F4FDA012C9150
:100EC000CC57DF4F8881C458D040820F912D911D9F
:100ED000813891050CF44BC000E8021BF894FE0128
:100EE000E058FF4F208161E8C62ED12CCC0EDD1ECC
:100EF000D6018C91821730F4DA018C91B22FB81B95
:100F00008B2F02C0822F800F80837894F60180811E
:100F100032E8E32EF12CEC0EFD1E281790F4112779
:100F2000822F9927AC01BE01C8018C0F9D1F0E9422
:100F30000F15D7018C91FE01E80FF11DCF01A8011B
:100F400009C0D7018C91281B3327FE01E80FF11D42
:100F5000CF01A901BC01CE010E940F15FE01EE5781
:100F6000FF4FD6018C919081891B8C93108220E0D9
:100F700030E0DE01AF57BF4F8C918F5F8C93AE0195
:100F80004E575F4FFA019081082F091B87FD1C9275
:100F9000CC57DF4F8881C458D040081709F5CD578A
:100FA000DF4F8881C358D0408B1561F49E01290F13
:100FB000311DFE01EB57FF4F808191810196918396
:100FC000808306C0FE01E957FF4F80818F5F8083D9
:100FD0008C91DA018C932115310511F0C90109C0FA
:100FE000FE01ED57FF4F80818B2580831FCF80E06E
:100FF00090E0DF91CF911F910F91FF90EF90DF90E4
:10100000CF90BF90089580E090E008951F920F92D6
:101010000FB60F9211248F939F9381EE86BD80911E
:1010200017018F5F80931701809119018F5F809363
:101030001901843638F010921901809118018F5FE0
:10104000809318018091150190911601892B49F028
:10105000809115019091160101979093160180934C
:1010600015019F918F910F900FBE0F901F901895B3
:1010700081EE86BDA89A80916E00816080936E009B
:1010800085B5887F846085BD08950F93FC017FB787
:10109000F894002359F080911C0190911D019683D2
:1010A0008583F0931D01E0931C010AC080911A0111
:1010B00090911B0196838583F0931B01E0931A01A5
:1010C000608354834383328321837FBF0F910895CC
:1010D000FC0160830895909316018093150180911F
:1010E000150190911601892BD1F708950F931F9345
:1010F000CF93DF938FB7F8941091170110921701D7
:1011000000911801109218018FBF112301F18091F5
:101110001C0190911D01892BD1F011501F3FB9F096
:10112000C0911C01D0911D012097B9F388818823BB
:1011300051F081508883882331F4EB81FC818981CF
:101140009A81099588830D80DE81C02DEDCF002323
:1011500011F180911A0190911B01892BE1F001504E
:101160000F3FC9F0C0911A01D0911B01209789F05F
:101170008881882351F081508883882331F4EB8162
:10118000FC8189819A81099588830D80DE81C02D3B
:10119000EDCF015038F7DF91CF911F910F91089556
:1011A0009927807F90708032910561F0813291059E
:1011B0001CF4409721F00CC0C09739F009C085E2BB
:1011C00090E0089588E290E008958BE290E0089521
:1011D00080E090E008959927807F9070803291059B
:1011E00061F0813291051CF4409721F00CC0C0974A
:1011F00039F009C084E290E0089587E290E0089514
:101200008AE290E0089580E090E008959927807F39
:1012100090708032910561F0813291051CF4409705
:1012200021F00CC0C09739F009C083E290E0089526
:1012300086E290E0089589E290E0089580E090E0F1
:101240000895CF93C82F0E940609FC01892B19F439
:101250008FEF9FEF13C08081282F33278C2F992782
:101260008770907002C0359527958A95E2F7C9017D
:101270008170907020FF02C081E090E0CF910895CE
:101280000F931F93CF93DF93182F062F0E94D00840
:10129000EC01812F0E94EB08FC011770209709F4E4
:1012A0004CC0202F332721303105D9F022303105B1
:1012B0001CF4232B41F041C02230310501F12330D1
:1012C000310561F13AC081E090E002C0880F991FBA
:1012D0001A95E2F72881282B28832081282B208348
:1012E0002CC002C0220F331F1A95E2F7922F90955F
:1012F0008881892388838081822B80831EC021E09E
:1013000030E002C0220F331F1A95E2F7922F90951A
:101310008081892380838881822B0EC081E090E0C8
:1013200002C0880F991F1A95E2F7982F9095808137
:1013300089238083888189238883DF91CF911F91BE
:101340000F910895CF92DF92EF92FF920F931F9328
:10135000CF93DF93D82E7B01C42EDB011C91012F8C
:10136000007F812F0E94D008EC01812F0E94EB08A2
:10137000FC0160E0209709F44AC0762F6D15E8F46F
:10138000402F552701E010E0D7018C91282F3327FB
:10139000C901807F907048175907C9F527703070D0
:1013A000C80102C0880F991F2A95E2F7682B08949C
:1013B000E11CF11C7F5F7D1538F3962F90954C2D25
:1013C00055274130510581F0423051051CF4452B21
:1013D00041F01DC04230510571F04330510589F094
:1013E00016C08881862B02C08881892388838081EA
:1013F000862B80830CC08081892380838881862B03
:1014000005C0808189238083888189238883DF9137
:10141000CF911F910F91FF90EF90DF90CF900895A3
:101420009927AA27BB27DC0199278827BC01CD0172
:101430002EEF31E040E050E00E944715DA01C9018B
:101440008D5C9C4C08959C0144275527CA01B90125
:1014500020E43FE140E050E00E941C159B01AC01FC
:10146000DC01CB01880F991FAA1FBB1F820F931F9E
:10147000A41FB51FCD01AA27BB27089581E0809343
:101480003E010895CF93DF93CFE1D1E023E080E0E8
:1014900090E0DC01A050B0400E947115F983E88310
:1014A00028962150029627FFF4CFDF91CF9108951F
:1014B0008093010108959B019927880F991F845AF1
:1014C0009D4F42E050E0BC01C9010E940215089501
:1014D0001F93CF93DF93142FC82FDD27E3E0CC0FAA
:1014E000DD1FEA95E1F7C25EDE4F843008F5862FF6
:1014F0000E94100A9C019C838B83412F55275E8399
:101500004D8389819A812817390730F488279927D4
:10151000841B950B9E838D838D819E8174E0880F43
:10152000991F7A95E1F79E838D831F8281E08883DE
:10153000DF91CF911F910895CF93DF93CDB7DEB7A1
:1015400022970FB6F894DEBF0FBECDBF282F843090
:1015500010F59927FC01A3E0EE0FFF1FAA95E1F714
:10156000E25EFE4F1082DC01A80FB91FA050B04010
:10157000818192810C010E948215BE016F5F7F4FB5
:10158000822F0E945B0A63E08A810E94400961E029
:1015900089810E94400922960FB6F894DEBF0FBEE3
:1015A000CDBFDF91CF9108950F931F93082F11277F
:1015B000B3E0000F111FBA95E1F7025E1E4F862FB0
:1015C0000E94100AF801948383831F910F9108955C
:1015D0000895DF92EF92FF920F931F93CF93DF93C3
:1015E000CDB7DEB722970FB6F894DEBF0FBECDBFE2
:1015F000809102018F3F51F480913E01882309F4CC
:10160000BCC01092020110923E01B7C0BE016F5FD4
:101610007F4F0E945B0A70910201072F112783E020
:10162000000F111F8A95E1F7025E1E4FF8018081BD
:10163000882309F498C0A381B48125813681AD0146
:10164000421B530BF780FF2009F050C099278230CE
:101650009105C1F0833091051CF4019739F049C020
:1016600083309105B9F00497D9F143C06F2D89817A
:101670000E94400961E08A810E94400982E0F801ED
:10168000808337C084E1F801878383E080836F2DF6
:10169000872F1BC0F801818192811216130624F452
:1016A00048175907A8F403C08417950788F4F80170
:1016B000B283A183809101018823D9F084E18783DB
:1016C00084E0808361E0809102010E947B1111C05F
:1016D000F80181819281820F931F9283818309C0D7
:1016E000872F0E949C0AF801F08203C0FA94F80147
:1016F000F782F8018081992703970297A0F501816D
:101700001281DA80F89460E08D2D0E944009E0900B
:101710008400F09085007894C8010E94230ABC01DF
:101720009C0144275527205A30404040504080912A
:101730008400909185008E199F09AA27BB278217E4
:101740009307A407B5079CF3F894809184009091C7
:1017500085008E199F0986179707B8F361E08D2DD4
:101760000E9440097894809102018F5F809302016A
:10177000843019F48FEF8093020122960FB6F8940B
:10178000DEBF0FBECDBFDF91CF911F910F91FF90B4
:10179000EF90DF900895CF93DF93CDB7DEB7289712
:1017A0000FB6F894DEBF0FBECDBFFC018081853E31
:1017B000B1F48181803199F482818F3781F4838102
:1017C0008F3769F484818F3751F485819927807F21
:1017D00090708034910519F48285807F19F080E043
:1017E00090E037C0BE016F5F7F4FCF010E94A50F11
:1017F00089818D3019F08FEF9FEF2BC08F81813061
:1018000019F08EEF9FEF25C08A81843019F4888506
:10181000882319F08DEF9FEF1CC08D81282F33276F
:1018200022FF06C08C81853019F08CEF9FEF11C02C
:1018300020FF0DC08B81813051F021FD03C08BEF63
:101840009FEF07C0823018F08AEF9FEF02C081E05F
:1018500090E028960FB6F894DEBF0FBECDBFDF91A3
:10186000CF9108958091400190914101A091420152
:10187000B09143010196A11DB11D80934001909349
:101880004101A0934201B093430181E090E00895AB
:101890000F9301E02FE331E042E35CE0602F84E44A
:1018A00091E00E9445080F910895F89480914001BD
:1018B00090914101A0914201B09143017894BC0103
:1018C000CD010895CF93DF93EC0188819981AA819E
:1018D000BB810097A105B10519F48FEF9FEF27C0D9
:1018E0000E94550C288139814A815B8162177307F8
:1018F0008407950750F4261B370B480B590B2E5FB6
:101900003F4F4F4F5F4750F00CC0621B730B840B6F
:10191000950B6E5F7F4F8F4F9F4718F081E090E0EF
:1019200006C0188219821A821B8280E090E0DF9143
:10193000CF910895EF92FF920F931F93CF93DF9370
:10194000EC017A018B01411551056105710529F002
:101950000894E108F108010911090894E11CF11C3F
:10196000011D111D8EEFE8168FEFF8068FEF0807A7
:101970008FE7180740F08DEFE82E8FEFF82E8FEFEE
:10198000082F8FE7182F89EEE81683E0F80680E02D
:10199000080780E0180728F00894E11CF11C011DDD
:1019A000111D0E94550C6E0D7F1D801F911F6883B5
:1019B00079838A839B83611571058105910541F4C3
:1019C0006F5F7F4F8F4F9F4F688379838A839B839D
:1019D000DF91CF911F910F91FF90EF900895FC013F
:1019E000892BA1F080819181A281B3810097A1050B
:1019F000B10561F04F5F5F4F6F4F7F4F4F3F2FEF4C
:101A000052072FEF62072FE3720718F08FEF9FEF57
:101A10000895480F591F6A1F7B1F408351836283BB
:101A20007383411551056105710541F44F5F5F4FA7
:101A30006F4F7F4F408351836283738380E090E0D8
:101A40000895FC0110821182128213820895CF93AF
:101A5000DF93CDB7DEB724970FB6F894DEBF0FBE85
:101A6000CDBFAA27BB27AC01BD01CE0101960E94C4
:101A70009A0CCE0101960E94620C8823D1F724961D
:101A80000FB6F894DEBF0FBECDBFDF91CF910895A2
:101A900020E030E0E8E6F2E081918A3A31F42F5F0D
:101AA0003F4F85E0E030F807B8F3C90108950F9380
:101AB0001F93CF93DF93CDB7DEB768970FB6F89437
:101AC000DEBF0FBECDBF809166028823D9F185EEBF
:101AD000898390E19A83809167028B8387E48C836A
:101AE00082E08D839E839B870E94280F9A8B898B2F
:101AF0008DE091E09C8B8B8B04E010E01E8B0D8BB6
:101B000083E090E00E94360F8F8BC8010E94360F51
:101B1000888FBE016F5E7F4FCE0101960E94C70F76
:101B20008F896AE00E943B15892F825D682FCE0164
:101B300001960E942D06833019F082E090E004C0E7
:101B40001092660280E090E068960FB6F894DEBFCF
:101B50000FBECDBFDF91CF911F910F910895482FF8
:101B600065E684EB0E94F604992708951F93CF93AE
:101B7000DF93EC01162F112371F0CE010E949C0F10
:101B8000882331F48AE20E94AF0D80E090E005C026
:101B900021961150F0CF81E090E0DF91CF911F911D
:101BA0000895EF92FF920F931F93CF93DF93CDB7DA
:101BB000DEB728970FB6F894DEBF0FBECDBF7C010D
:101BC000FC018181803109F034C18081853E09F0BA
:101BD00030C18481823009F02CC1838199278C0126
:101BE0000074107086FD25C185819927807F9070D3
:101BF000409709F01EC182859927807F9070409799
:101C000009F017C1BE016F5F7F4FC7010E94A50F8A
:101C1000F7018381873049F0893039F00E94280F1D
:101C200029813A8128173907A9F5F7018381082FFF
:101C300011270630110509F47AC00730110594F414
:101C40000230110571F10330110524F40130110542
:101C5000D1F0CCC00330110569F10530110509F44C
:101C600047C0C4C00830110509F488C00830110508
:101C70000CF47AC00930110509F496C00F30110533
:101C800009F4BAC0B3C061E08B819C810E94B60D9B
:101C9000882311F4C801CFC06D818B819C810E9483
:101CA000770F61E08B819C810E94B60D882309F437
:101CB000A0C018C061E08B819C810E94B60D882372
:101CC00009F497C08B819C810E94360F2E81922F40
:101CD000909598238D818223982B692F8B819C81ED
:101CE0000E94770F8B819C810E94360F8D8384C068
:101CF00064E08B819C810E94B60D882309F479C031
:101D00006D818B819C810E94770F8B819C816E817C
:101D100001960E94770F8B819C816F8102960E94B1
:101D2000770F8B819C81688503960E94770F64E012
:101D30008B819C810E94B60D882309F45AC08B8147
:101D40009C810E94360F8D838B819C8101960E941D
:101D5000360F8E838B819C8102960E94360F8F8373
:101D60008B819C8103961CC0F7018281809367025E
:101D700081E08093660282E090E05DC00E94280FBF
:101D80009A8389838DE091E09C838B8304E010E04B
:101D90001E830D8383E090E00E94360F8F83C8017D
:101DA0000E94360F888728C08B819C818D5091407E
:101DB00009F03FC00D811E8104301105D1F583E08B
:101DC00090E00E94360F9F81891799F5C8010E9403
:101DD000360F9885891769F589819A810E942E0F9F
:101DE000892B51F08CE20E94AF0D23C08BE20E9440
:101DF000AF0D81E090E01FC0BE016F5F7F4FC70154
:101E00000E94C70FF701838180648383C7010E940A
:101E1000C304F70183818F3461F488E190E028E006
:101E20000FB6F894A895809360000FBE20936000D1
:101E3000FFCF80E090E028960FB6F894DEBF0FBE8B
:101E4000CDBFDF91CF911F910F91FF90EF9008953B
:101E5000A8E0B0E00E947115CF010895A8E0B0E0BD
:101E60000C010E94821580E090E008958430910575
:101E7000E9F08530910550F48230910589F0833086
:101E8000910588F48130910589F122C08630910551
:101E9000B9F08630910588F087309105A9F018C017
:101EA00085E090E00895ABE0B0E002C0AAE0B0E0C9
:101EB0000E946915802D9927089581E090E008958A
:101EC000EEEFFFE38491F7CFEFEFFFE38491F3CFE1
:101ED00021E0843F920718F080E090E00895DC0153
:101EE000AC5FBF4F0E946915802D992708958330FC
:101EF000910521F08430910521F00BC0ABE0B0E0FA
:101F000002C0AAE0B0E0062E0E94761580E090E0C4
:101F100008958830910520F021E0843F920718F061
:101F20008FEF90E00895DC01AC5FBF4F062E0E945A
:101F3000761580E090E0089520E030E0845F9140E5
:101F400010F421E030E0C9010895CF93DF939C01A4
:101F500051E0D9011696E901259640E0FB019C91DC
:101F600090838881852311F090689083433031F409
:101F700051E0D9011B96E9012A9602C0550F11962E
:101F80004F5F3196483058F3DF91CF910895CF934A
:101F9000DF939C0151E0D9011696E901259640E0B6
:101FA000FB0180818F778C93808187FF03C08881BC
:101FB000852B8883433031F451E0D9011B96E90128
:101FC0002A9602C0550F11964F5F3196483048F35C
:101FD000DF91CF9108950F931F93CF93DF9300E08C
:101FE00010E0C8E6D0E0FE018491682FC8010E948D
:101FF000770F0F5F1F4F2196F1E0043F1F079CF3FF
:1020000080E090E0DF91CF911F910F9108950895A6
:1020100008958F929F92BF92CF92DF92EF92FF929C
:102020000F931F93CF93DF93E0E0F0E021E0822E47
:10203000912CA2E0B0E094E0C92ED12C08E010E091
:1020400030910B012091C001B0906901BF01AF0137
:102050008AE6E82E81E0F82EE7018881C9E0D0E029
:10206000EC0EFD1E882331F53230B9F4E330F10572
:102070000CF090C0C401042E02C0880F991F0A946E
:10208000E2F780952823CD01042E02C0880F991F06
:102090000A94E2F78095282325C0313009F07AC0F0
:1020A000C401062E02C0880F991F0A94E2F780959A
:1020B000282334C0BB20A1F5323029F5E330F105E7
:1020C0000CF068C0C401042E02C0880F991F0A9446
:1020D000E2F7282BCD01042E02C0880F991F0A9425
:1020E000E2F7282BC601042E02C0880F991F0A941C
:1020F000E2F780952823C801042E02C0880F991F9B
:102100000A94E2F745C0313009F044C0C401062EFC
:1021100002C0880F991F0A94E2F7282BCD0132C024
:10212000323029F5E330F10514F5C601042E02C062
:10213000880F991F0A94E2F7282BC801042E02C0C9
:10214000880F991F0A94E2F7282BC401042E02C0BD
:10215000880F991F0A94E2F780952823CD01042E59
:1021600002C0880F991F0A94E2F780952823313026
:1021700089F4CD01062E02C0880F991F0A94E2F758
:10218000282BC801062E02C0880F991F0A94E2F777
:102190008095282331964C5F5F4F6E5F7F4FE43010
:1021A000F1050CF459CF2093C0010E94BB01DF91CF
:1021B000CF911F910F91FF90EF90DF90CF90BF9044
:1021C0009F908F900895CF93DF9320E030E080912F
:1021D000BC01882351F427E030E02150304037FF24
:1021E000FCCF81E0809373012EC0E901C959DE4F15
:1021F0008B81813011F58091BD01282F332727FD78
:1022000030958C819D81820F931F2091B601309172
:10221000B701281739078CF01B8268816F77888196
:102220009981880F892F881F990B482F4F708A81B9
:102230008111406281EB0E94F604299681E0C63A42
:10224000D807B1F2ACF20E940910DF91CF91089546
:10225000833011F40E94E31080E090E00895EF9243
:10226000FF921F93CF939927009719F0019749F098
:102270003BC010E0812F0E949C0A1F5F1430D0F3F6
:1022800033C00E94E90AC0E087E6E82E81E0F82E1C
:10229000F70183818823F9F08281992787FD909542
:1022A000009719F0049749F014C08C2F0E948314F2
:1022B000182F8C2F0E946F1407C08C2F0E9483143C
:1022C000182F8C2F0E947914412F682F8C2F0E9479
:1022D000680AF7011382CF5F89E090E0E80EF91EEB
:1022E000C430B0F20E94E01480E090E0CF911F91E2
:1022F000FF90EF9008950F931F93CF93082F162F01
:10230000C0E09927FC0123E0EE0FFF1F2A95E1F7BB
:10231000E80FF91FE959FE4F8281843009F4C1E0CA
:10232000412F6C2F808191810E940713112321F08E
:102330006C2F802F0E94B314CF911F910F9108959D
:10234000089508950F931F93CF93DF93C9E6D1E0CB
:1023500000E510E0C8010E94360F888329960F5FC0
:102360001F4F81E0CF39D807A9F3A4F3DF91CF91B4
:102370001F910F9108955F926F927F928F929F921B
:10238000AF92BF92CF92DF92EF92FF920F931F9383
:10239000CF93DF93EC019924FC0163E0EE0FFF1F64
:1023A0006A95E1F7E80FF91FE959FE4F62808C59F1
:1023B0009F4F0E94360FC82EC694C694C694C694EA
:1023C0005FE0F52EF8222EE02C1508F4E6C0FF2081
:1023D00009F4E3C038E03F1508F4F32ECE0182592A
:1023E0009F4F0E94360F782E76947694769476944A
:1023F0004FE0842E882286E790E00E94360F9927CE
:102400000C2E02C0959587950A94E2F780FF03C0D1
:1024100031E0532E01C0592C87E790E00E94360F1F
:1024200099270C2E02C0959587950A94E2F780FFB4
:1024300003C021E0922E01C0992483E290E0C89F5E
:102440009001C99F300DD89F300D1124C901C62DB0
:10245000DD279E012F713070820F931F88589F4F88
:102460000E94360F082F1127C80180579E4F0E94E7
:10247000360FE82EC8018E539E4F0E94360FE0E0C3
:10248000F0E0AF2DBB27EA17FB07DCF591E0A92EA2
:10249000B12C0E2D1127E82EFF24D090BB012091E6
:1024A0004B0130914C016C2D7727A501062E02C0FF
:1024B000440F551F0A94E2F7CA018095909528238E
:1024C0003923C8010E2E02C0959587950A94E2F72C
:1024D00080FF0DC0C7010E2E02C0959587950A9406
:1024E000E2F780FF02C0DD2011F0242B352B31965E
:1024F0006F5F7F4FEA17FB07C4F230934C012093C4
:102500004B013EE0381520F141E050E002C0440F9D
:10251000551F8A94E2F7CA018095909520914B014E
:1025200030914C012823392330934C0120934B01E7
:10253000CF71D070219761F4552021F08091BB01BB
:10254000882331F0242B352B30934C0120934B0101
:102550008EE0871510F141E050E002C0440F551F96
:102560007A94E2F7CA018095909520914B013091C1
:102570004C012823392330934C0120934B0165FEF5
:102580000CC0992021F08091BB01882331F0242BCD
:10259000352B30934C0120934B01DF91CF911F914C
:1025A0000F91FF90EF90DF90CF90BF90AF909F90F2
:1025B0008F907F906F905F900895CF93DF93C0E0EE
:1025C000D0E0CE010E94BB112196C730D105CCF3DB
:1025D00080914B018093C00180914B0190914C01FF
:1025E000892F99278093C1010E94BB01DF91CF9170
:1025F00008959927009719F0039721F005C00E94CC
:10260000A21102C00E94DD1280E090E00895242F04
:10261000382F3F77880F892F881F990B9195482F66
:102620004F704064222329F0662311F0406201C0FC
:102630004061632F81EB0E94F6040895FC018281C2
:1026400086FF13C08381813081F49481992369F4DA
:102650004581442339F08681880F682F892F0E9495
:10266000680A0895842F0E949C0A08951F93CF93AF
:10267000182FC62F80915B0180FF11C0812F0E940F
:10268000FB13682F6F77880F892F881F990B482FAE
:102690004F704066C111406182EB0E94F604809148
:1026A0005B0183FF04C06C2F812F0E942414CF9103
:1026B0001F910895EF92FF920F931F93CF93DF9393
:1026C0008DE491E00E94620C813009F44BC08DE2F0
:1026D00090E00E94360F80935B0142E350E060E09F
:1026E00070E08DE491E00E949A0C00E0EE24FF245B
:1026F000C1E5D1E018E2F701EC59FD4F84910E9449
:102700002109992787FD9095009791F0019719F578
:10271000988193333CF089818230E9F082E08983AB
:1027200061E00FC080915B0184FD15E0910F12C044
:1027300098819E3C54F48981813069F081E08983DD
:1027400060E0802F0E94361306C080915B0185FDFA
:1027500015E0911B98830F5F0894E11CF11C2296F1
:10276000053040F2DF91CF911F910F91FF90EF90D4
:102770000895FF920F931F938B010E94360FF82E3E
:10278000C8010E94360F682F82958F70282F33273B
:1027900088EE93E0289FA001299F500D389F500D8F
:1027A0001124862F99278F70907024E630E0829F45
:1027B000B001839F700D929F700D1124460F571F1B
:1027C0008F2D82958F70282F3327C90163E0880FE2
:1027D000991F6A95E1F7820F931F820F931F480F8D
:1027E000591F8F2D99278F709070840F951F1F91FF
:1027F0000F91FF90089599278130910589F08230DB
:1028000091051CF4892B39F01CC08230910579F0B8
:10281000039791F016C064E270E085E290E004C096
:1028200066E270E087E290E00E94B913089568E2E2
:1028300070E089E290E0F8CF6AE270E08BE290E02D
:10284000F3CF8FEF9FEF089599272091B601309134
:10285000B701662369F0FC0153E0EE0FFF1F5A95A4
:10286000E1F7E80FF91FE959FE4F84E082830BC0BE
:10287000FC0143E0EE0FFF1F4A95E1F7E80FF91F57
:10288000E959FE4F6283178216823583248381E0E3
:1028900083830895282F3327662371F0F90173E0AD
:1028A000EE0FFF1F7A95E1F7E20FF31FE959FE4F94
:1028B0008281843089F00DC0F90163E0EE0FFF1FC3
:1028C0006A95E1F7E20FF31FE959FE4F82818823F1
:1028D00019F081E090E0089580E090E00895992754
:1028E000880F991F880F991FC2960E94360F99274B
:1028F00008959927880F991F880F991FC3960E94E2
:10290000360F992708959927880F991F880F991FC7
:10291000C4960E94360F992708959927880F991F0A
:10292000880F991FC2960E94770F0895262F992726
:10293000880F991F880F991F622FC3960E94770FE7
:102940000895E82FFF27662329F0EE0FFF1FED5FA4
:10295000FE4F04C0EE0FFF1FEC5FFE4F642F80811F
:102960000E94400908951F93CF93C82F162F8230DD
:1029700020F59927FC01EE0FFF1FEE0FFF1FE80F58
:10298000F91FE45AFE4F608360E0112309F461E00F
:1029900041E08C2F0E94A11440E0612F8C2F0E94F7
:1029A000A11485E0C89FC001112444EF51E060E00C
:1029B00070E0835A9E4F0E949A0CCF911F91089508
:1029C000FF920F931F93CF93DF93FF24CCE5D1E0C9
:1029D0008E010F5F1F4FC8010E94620C882329F4EB
:1029E00041E068818F2D0E94A114F3940B5F1F4F6B
:1029F000259681E08F1578F7DF91CF911F910F9188
:102A0000FF900895FB01DC0140FF05C002C0059066
:102A10000D9205900D9242505040C8F70895FB0169
:102A2000DC0140FF05C002C001900D9201900D92A3
:102A300042505040C8F70895629FD001739FF00143
:102A4000829FE00DF11D649FE00DF11D929FF00D3E
:102A5000839FF00D749FF00D659FF00D9927729F75
:102A6000B00DE11DF91F639FB00DE11DF91FBD0100
:102A7000CF0111240895991B79E004C0991F96177E
:102A800008F0961B881F7A95C9F780950895A1E2F2
:102A90001A2EAA1BBB1BFD010DC0AA1FBB1FEE1FD8
:102AA000FF1FA217B307E407F50720F0A21BB30B23
:102AB000E40BF50B661F771F881F991F1A9469F79F
:102AC00060957095809590959B01AC01BD01CF01FB
:102AD0000895F999FECFB2BDA1BDF89A119600B440
:102AE0000895F7DFE02DF5DFF02D0895F999FECF79
:102AF000B2BDA1BD00BC11960FB6F894FA9AF99A2E
:0E2B00000FBE0895F3DF012CF1DF11240895BC
:082B0E00FF01FF16143734002B
:00000001FF
